:103E480000010C01010402011E030A960401320557
:103E5800030306006407010108000009015A0E0166
:103E6800010F000112006413010114013C1501FA4D
:103E78001664FA17FFFF1D00072000072400022719
:103E880001012F013C30010132010335FFFF3603E8
:103E9800073CFFFF3DFFFF180002191E461A0002EB
:103EA8001B00022D32C82E0001FAFAFA1800001978
:103EB800FFFF1A00001B00002D32C82E0001FAFA7D
:103EC800FA18000019FFFF1A00001B00002DFFFF61
:063ED8002EFFFFFAFAFACA
:10004800900786E0FEA3E0FF7457BE0010D39F40E0
:100058000C903E4812001EE493F599804C900014D1
:10006800E0D394044014900786E0FEA3E0FF903E9E
:100078004812001EE493F599802F900014E0D39461
:10008800034014900786E0FEA3E0FF903E5D120057
:100098001EE493F5998012900786E0FEA3E0FF9096
:1000A8003E7212001EE493F59990078612000E9096
:1000B8000786E0FEA3E0FF746C6F4E7003751300B3
:1000C80022900072E0B402087401900072F0D20C21
:1000D80090013AE090002AF090013BE090002BF06C
:1000E80090013CE090002CF0A20AB3401690013A2F
:1000F800E0700C90013BE0700690013CE0600280EB
:1001080002C20A90013AE0B4300F90013BE0B447D4
:100118000890013CE0643B60028004D20B8002C27C
:100128000BE557B40102800302024B900057E0F53B
:1001380065900062E0F567900063E0F568900074F0
:10014800E0F56990007AE0900029F090007CE0F5F5
:100158006490007DE0F566900080E0F56390008192
:10016800E0F562900090E0900041F0900091E090FE
:100178000042F0900092E0900043F0900093E090ED
:100188000044F0900094E0900045F0900095E090D5
:100198000046F0900096E0900047F0900097E090BD
:1001A8000048F0900099E0900033F090009AE090B9
:1001B8000034F090009BE0900035F090009CE090B7
:1001C8000036F0900079E0B4011790000A740FF03F
:1001D800A374FFF090000CE4F0A3F074029000798F
:1001E800F0900079E0B4035990000CE0FEA3E0FF22
:1001F80090000AE0FCA3E0FD1200037410123F5DBA
:100208007408123F4FEF900026F0EF700674FF90CD
:100218000026F07400900079F090000BE090002721
:10022800F090000AE0900028F0900026E0900789FE
:10023800F0900027E090078AF0900028E090078B64
:10024800F0803F900081E07006755701756200A24A
:100258000AB3402E90013AE090002AF090013BE06A
:1002680090002BF090013CE090002CF090002AE0E8
:10027800700C90002BE0700690002CE06002800269
:10028800C20AE5657003756502E567700375670264
:100298007E887F75E5658E048F05FF123F3F8C3899
:1002A8008D39E56875F0FAA4FFAEF0E5678E048F26
:1002B80005FF123F3F8C3C8D3D90004FE0F55F906D
:1002C800004DE0FE900069E0B5061890004CE0FE95
:1002D800900068E0B5060C90004BE0FE900059E0F5
:1002E8006E606F900069E07006900068E0600674C8
:1002F80000900059F0900069E0B402089000497439
:1003080001F08005900049E4F0900068E0B402082C
:1003180090004A7401F0800590004AE4F09000686B
:10032800E0600690004AE060028005755F03800384
:10033800755F04E558B55702D20C900068E090004C
:100348004CF0900069E090004DF0900059E090006A
:100358004BF0740190009EF0740190009FF07400BF
:100368009000A0F074009000A1F074009000A2F03A
:1003780074009000A3F074009000A4F07401900041
:10038800A5F074019000A6F074019000A7F0740025
:100398009000A8F074009000A9F074009000AAF0F2
:1003A80074009000ABF074019000ACF07401900000
:1003B800ADF074009000AEF074009000AFF07400DF
:1003C8009000B0F074009000B1F074009000B2F0AA
:1003D8007401900362F07401900363F07400900359
:1003E80064F07400900365F07400900366F0740084
:1003F800900367F07400900368F074009003A2F013
:1004080074019003A3F074009003A4F074009003A7
:10041800A5F074009003A6F074009003A7F0740090
:100428009003A8F074009003E2F074009003E3F0E6
:1004380074009003E4F074009003E5F074009003F6
:10044800E6F074009003E7F074009003E8F074019C
:10045800900422F07400900423F07400900424F0B7
:100468007400900425F07400900426F07400900441
:1004780027F07400900428F022E5B554F7F5B5E5A7
:10048800B554FDF5B5C292C287C290C207E5B5540E
:10049800FBF5B5755004E55004F55190004FE0F5B3
:1004A8005F900025E4F0C209E5B554FEF5B5227564
:1004B8000A00750900AE09AF0A7457BE00039F50C1
:1004C80003020574903E4812001EE49390004E12F9
:1004D8003F750FBF00010EE0FC903E4812001EEC75
:1004E800FEE493FFEEC39F5026AE09AF0A0FBF008C
:1004F800010E903E4812001EAE09AF0AE493FC902C
:100508003E4812001EE49390004E123F75ECF0AE88
:1005180009AF0A903E4812001EE49390004E123F25
:1005280075E0FC903E4A12001EECFCE493FDECD30F
:100538009D4019903E4A12001EE493FC903E4812DA
:10054800001EE49390004E123F75ECF0AE09AF0A1E
:1005580074022FFF50010E8E098F0A780A74012643
:10056800F6500418E436F640030204BD22750A006A
:10057800750900AE09AF0A7415BE00039F50030247
:100588000642903E9F12001EE49390004E123F7563
:100598000FBF00010EE0FC903E9F12001EECFEE42F
:1005A80093FFEEC39F5026AE09AF0A0FBF00010E9E
:1005B800903E9F12001EAE09AF0AE493FC903E9F46
:1005C80012001EE49390004E123F75ECF0AE09AF96
:1005D8000A903E9F12001EE49390004E123F75E071
:1005E800FC903EA112001EECFCE493FDECD39D4070
:1005F80019903EA112001EE493FC903E9F12001E2B
:10060800E49390004E123F75ECF0AE09AF0A740FF8
:100618006F4E7006750A15750900AE09AF0A7402A7
:100628002FFF50010E8E098F0A780A740126F650A2
:100638000418E436F6400302057B22750A007509A2
:1006480000AE09AF0A7415BE00039F5003020710DD
:10065800903EB412001EE49390004E123F750FBFF7
:1006680000010EE0FC903EB412001EECFEE493FF85
:10067800EEC39F5026AE09AF0A0FBF00010E903E91
:10068800B412001EAE09AF0AE493FC903EB4120007
:100698001EE49390004E123F75ECF0AE09AF0A903D
:1006A8003EB412001EE49390004E123F75E0FC9099
:1006B8003EB612001EECFCE493FDECD39D4019906D
:1006C8003EB612001EE493FC903EB412001EE49362
:1006D80090004E123F75ECF0AE09AF0A740F6F4EE2
:1006E8007006750A15750900AE09AF0A74022FFF66
:1006F80050010E8E098F0A780A740126F6500418E4
:10070800E436F6400302064922750A00750900AE70
:1007180009AF0A7415BE00039F50030207DE903E1E
:10072800C912001EE49390004E123F750FBF0001DE
:100738000EE0FC903EC912001EECFEE493FFEEC3EF
:100748009F5026AE09AF0A0FBF00010E903EC91296
:10075800001EAE09AF0AE493FC903EC912001EE4E5
:100768009390004E123F75ECF0AE09AF0A903EC967
:1007780012001EE49390004E123F75E0FC903ECBB1
:1007880012001EECFCE493FDECD39D4019903ECB87
:1007980012001EE493FC903EC912001EE4939000E0
:1007A8004E123F75ECF0AE09AF0A740F6F4E70062B
:1007B800750A15750900AE09AF0A74022FFF5001BA
:1007C8000E8E098F0A780A740126F6500418E4364A
:1007D800F6400302071722054C22054B22054DC29D
:1007E800CF2290F800E4936406600280FE758401CD
:1007F80075A70075FF80900788E4F075C91075A784
:100808000F75A1C775A70075D90075CEFF75A70F1D
:1008180075F1FE75F2FF75F33775F47875A4BA753E
:10082800A5FF75A60775AE0075AFFF75D48175D5A0
:10083800FF75D6FF75D7FFC293C294C291E5B55430
:10084800BFF5B5E5B554DFF5B5E5B554EFF5B5E554
:10085800B5547FF5B5E5B554F7F5B5E5B554FDF5EF
:10086800B575A70075A20175A14775F80975BC0192
:1008780075BE0475BD6C75BE0775BDA075BE0875DF
:10088800BD0175BC0075BB1875BC2075BA0875E844
:100898008075D11375A70F75E10575E20075C7401E
:1008A800759700759780740A123F2F7597C0E59762
:1008B8005420700280F8758F0275A700D2AF759822
:1008C8000075A90C75A70F75AB4375ADFB75AC1E0C
:1008D80075A700758911758E00758C00758A00D210
:1008E800A9D28C758D00758B00D2ABD28E75CD00D8
:1008F80075CC0075CA0075CB00D2ADC2CFD2CA750F
:1009080091047592007593CD75EF0675D94075CF32
:1009180001900786E4F0A3F0751300751400C299DE
:10092800D20A74C8F51875170012269075A70FE536
:10093800FB90001AF0E5FA90001BF0E5F990001C16
:10094800F075A70090F800E493F5081227C7122D58
:1009580001900789E0900026F090078AE090002730
:10096800F090078BE0900028F090078CE090002929
:10097800F090078DE0F56590078EE0F56790078F9A
:10098800E0F568900790E0F569900791E0F56490CC
:100998000792E0F566900793E0F563900794E0F519
:1009A80062900795E090002AF0900796E090002B5F
:1009B800F0900797E090002CF0900798E0900041A5
:1009C800F0900799E0900042F090079AE090004379
:1009D800F090079BE0900044F090079CE090004561
:1009E800F090079DE0900046F090079EE090004749
:1009F800F090079FE0900048F09007A0E090003347
:100A0800F09007A1E0900034F09007A2E090003544
:100A1800F09007A3E0900036F07400900082F09008
:100A2800013AE0700C90013BE0700690013CE060F8
:100A3800028004C20A8002D20A90F807E493900068
:100A480021F0900021E0440A900021F0900021E07C
:100A580054FE900021F07406900012F07402900089
:100A680013F090F802E493900014F07403900015CA
:100A7800F07403900016F0741A900017F074059043
:100A88000018F0900014E0B404067404900018F004
:100A9800900014E0B403067403900018F0740490F6
:100AA8000019F090F804E49390001DF07400900091
:100AB8001EF090F805E49390001FF090F806E49378
:100AC800900020F074FF900022F0745A900125F0F5
:100AD8007446900126F07420900127F07434900138
:100AE80028F07448900129F0745090012AF074326B
:100AF80090012BF0743490012CF0742090012DF0AB
:100B0800743590012EF0742D90012FF074539001DC
:100B180030F0746F900131F0746C900132F07420F1
:100B2800900133F090007AE0D3940140067400906D
:100B3800007AF0755701755801740390004CF01253
:100B480000C91204B7900014E0B4040512064380EB
:100B580011900014E0D39404400512057580031227
:100B680007111226BCE5B554FEF5B5900025E4F052
:100B7800900786E4F0A3F0752300752200754700FE
:100B880075290075280075480075310075300075A5
:100B98004900755300755400755900755004755116
:100BA8000175333C753200756F00756E007570CD38
:100BB80075550075560075420075430075440075FB
:100BC8004500755A00754600754100754000900053
:100BD80006E4F0A3F0900008E4F0A3F0755D00755A
:100BE8005E0090000E74FDF0A374E8F0900023E41A
:100BF800F07464900024F0C200D201C202D20375DE
:100C08004C00756C00C297C2A0C296C295C2A2C21F
:100C18000C7E017F00900028E0123F5D900027E0E5
:100C28002FFF50010E90000AEEF0A3EFF09000267F
:100C3800E0700674FF900026F090000AE0FEA3E042
:100C4800FFEFD394FFEE940F400790000AE4F0A35F
:100C5800F07400900071F07400900079F0740090C6
:100C68000082F0740090008DF074009000B4F0E5FC
:100C7800667003756604743A90074EF074FD900729
:100C88004FF09003D4E0900414F0D2B0D2B7D2A7BA
:100C9800D2A6D2B1D2A3C207A2B6B39204A2B3B36A
:100CA8009205D29CD2EC75CF01A298B34005C298A8
:100CB800123065E5136006A299B3B340028005C2FD
:100CC800991235DBE51464016005E514B40402806B
:100CD800D5E54CD39405400CE559C394C85002059A
:100CE80059754C00E570C394F0501A786E12003FA5
:100CF800AE6EAF6FEFD394E8EE94034008057075BD
:100D08006F00756E00C28E7E047F00E54B123F5D5A
:100D1800E58D75F004A4FDACF0EF2DFDEE3CFCE58F
:100D28008B75F04084FF7E00ED2FFFEC3EFE8E2495
:100D38008F25D28EA2B6300401B35003020E74A2DE
:100D4800B6300401B35003020E74A2B6405A0553DC
:100D5800E5B54401F5B5900024E4F0E553D3956575
:100D680040447C887D75123D678E228F23E5472F8E
:100D7800FF50010E7401123F4F8E228F23852347A7
:100D8800755301C28E758D00758B00754B00D28E20
:100D98007403BE00039F50069000257401F0E542DD
:100DA800B40603754200D204A2B6B35003020E740F
:100DB800C20490006BE0601812371CA200B3400810
:100DC800E5B54408F5B58006E5B554F7F5B58002F4
:100DD800C20090006EE06018123871A202B3400899
:100DE800E5B54402F5B58006E5B554FDF5B58006D0
:100DF800E5B554FDF5B5A207B34004D2968002C20A
:100E080096900059E06004D2958002C29590004AFD
:100E1800E0B40104D2978002C297900049E0B4017F
:100E280004D2A08002C2A0A209B34004D2A28002C8
:100E3800C2A2900018E0FE900014E0C39E40099002
:100E48000014E0D39408400974FB900023F01204C6
:100E58008190001DE0601590001DE0FE900017E0F5
:100E68006E600974FE900023F0120481C2CA7E01EC
:100E78007F00E54D123F5DE5CD2FFF50010E8E2618
:100E88008F27D2CAE564B4014890000EE0FCA3E0C5
:100E9800FDEFC39DEE9C4039B208E5294528601353
:100EA800A208B34008E5B54404F5B58006E5B55495
:100EB800FBF5B590000EE0FEA3E0FF900010E0FC0B
:100EC800A3E0FDEF2DFDEE3CFC90000EECF0A3ED51
:100ED800F0A2B3300501B35003020FB9A2B3300535
:100EE80001B35003020FB9A2B35003020FB2055465
:100EF800E5B54401F5B5900024E4F0E554D39567D1
:100F08005003020FB07CEA7D60AE26AF27123D6722
:100F18008E288F29E568123F5D74FF8E048F05FFC8
:100F2800123F3F8C288D29E5482DFD50010C740196
:100F38008C068D07123F4F8E288F29852948A209D4
:100F4800B340157464123F5D900067E08E048F050E
:100F5800FF123F3F8C288D2975540190000EE0FE4A
:100F6800A3E0FFAC26AD2712000390000EEEF0A31D
:100F7800EFF0E566FF123F3F740AFF123F3F900013
:100F88007BE08C068D07123F5D74148E048F05FF7D
:100F9800123F3F900010ECF0A3EDF0C2CA75CD00EF
:100FA80075CC00754D00D2CAD205A2B3B34002C2B7
:100FB80005900025E0B40107E555C39406400302F7
:100FC80015C5E56C90266FF8282873900059E0C382
:100FD80094024003021127E550D3940150030211F3
:100FE80027E55075F040A4FFAEF090031212001EE2
:100FF800E0C395445018E55075F040A4FFAEF0905A
:10100800031112001EE0F52D752C00021127E55082
:1010180075F040A4FFAEF090031012001EE0C395D7
:101028004440030210C3E55075F040A4FFAEF090B1
:10103800031112001EE55075F040A4FFAEF0E0FC6D
:1010480090030F12001EECFEE0FFEEC39FFEE5507A
:101058008E0475F040A4FFAEF090031012001EE05D
:10106800F40425448C0088F0A4FFAEF0E5508F040A
:101078008E0575F040A4FFAEF090031212001EE535
:101088005075F040A4FFAEF0E0FA90031012001E75
:10109800EAFEE0FFEEC39FFECDCCCD8E07123F3FA8
:1010A800E55075F040A4FFAEF090030F12001EE06B
:1010B8002DFD50010C8C2C8D2D8064E55075F04071
:1010C800A4FFAEF090030F12001EE55075F040A487
:1010D800FFAEF0E0FC90030E12001EECFEE0FFEE07
:1010E800C39F8544F0A4FFAEF0E5508F048E0575CC
:1010F800F040A4FFAEF090031012001EE0FECDCC2D
:10110800CD8E07123F3FE55075F040A4FFAEF0903A
:10111800030E12001EE02DFD50010C8C2C8D2D7538
:101128006C010215C5900059E0C3940240030212F5
:10113800DA90004FE0D395505003021283E55075C2
:10114800F040A4FFAEF090031812001EE0C39544CF
:101158005018E55075F040A4FFAEF0900317120048
:101168001EE0F52B752A00021283E55075F040A4A5
:10117800FFAEF090031612001EE0C3954440030230
:10118800121FE55075F040A4FFAEF090031712004F
:101198001EE55075F040A4FFAEF0E0FC9003151278
:1011A800001EECFEE0FFEEC39FFEE5508E0475F0D6
:1011B80040A4FFAEF090031612001EE0F40425448C
:1011C8008C0088F0A4FFAEF0E5508F048E0575F012
:1011D80040A4FFAEF090031812001EE55075F040D1
:1011E800A4FFAEF0E0FA90031612001EEAFEE0FF3C
:1011F800EEC39FFECDCCCD8E07123F3FE55075F074
:1012080040A4FFAEF090031512001EE02DFD500122
:101218000C8C2A8D2B8064E55075F040A4FFAEF04D
:1012280090031512001EE55075F040A4FFAEF0E0E3
:10123800FC90031412001EECFEE0FFEEC39F8544F1
:10124800F0A4FFAEF0E5508F048E0575F040A4FFC2
:10125800AEF090031612001EE0FECDCCCD8E071224
:101268003F3FE55075F040A4FFAEF0900314120024
:101278001EE02DFD50010C8C2A8D2BE550B4012267
:10128800E55FD39401401BE550C395555014E544E0
:10129800C39405500D90035FE0A828B8000695296F
:1012A80040028003755002E550B55F2290004FE080
:1012B800D395504019E55075F040A4FFAEF0900367
:1012C8001712001EE0A822B80006952340028002EB
:1012D800055F756C020215C5900059E0B4022AE555
:1012E8005075F040A4FFAEF090031712001EE0F511
:1012F8002B752A00E55075F040A4FFAEF090030E60
:1013080012001EE0F52D752C00900059E0B4030F73
:10131800900051E0F52B752A00752D00752C00758D
:101328006C030215C5E55075F040A4FFAEF09003BC
:101338002012001EE0C3955940030213FC90004997
:10134800E07036E550D394014029AE22AF23AC2C8F
:10135800AD2DEDD39FEC9E401AE55075F040A4FFEB
:10136800AEF090031E12001EE0A828B80005D39521
:10137800295002800215508034E550D39402402948
:10138800AE22AF23AC2CAD2DEDD39FEC9E401AE5D9
:101398005075F040A4FFAEF090031E12001EE0A8A6
:1013A80028B80005D39529500280021550E550C38E
:1013B800955F502FE550C395555028AE22AF23AC0A
:1013C8002AAD2BEFD39DEE9C4019E55075F040A453
:1013D800FFAEF090031F12001EE0A828B800069583
:1013E80029400280020550C290E55065516005C24F
:1013F80007755900756C040215C5E55075F040A4D1
:10140800FFAEF090031A12001EE0B40117E5507504
:10141800F040A4FFAEF090032012001EE0240AC39F
:10142800955940030214D2752F64752E00A207B394
:10143800500B900060E02405C3954440030214D289
:10144800E55075F040A4FFAEF090031D12001EE0B9
:10145800C395444064E55075F040A4FFAEF0900396
:101468001C12001EE55075F040A4FFAEF0E0FC90A1
:10147800031B12001EECFEE0FFEEC39F8544F0A4A0
:10148800FFAEF0E5508F048E0575F040A4FFAEF076
:1014980090031D12001EE0FECDCCCD8E07123F3FFB
:1014A800E55075F040A4FFAEF090031B12001EE05B
:1014B8002DFD50010C8C2E8D2FAE22AF23AC2EADFE
:1014C8002FEFD39DEE9C4002D207756C050215C51F
:1014D800E550B40109900059E0C394024003021595
:1014E800A5900358E0D3954450030215A5900356E0
:1014F800E0C395445040900357E0FE900355E0F454
:10150800042EFE900356E0F40425448E0088F0A4CF
:10151800FFAEF0900358E0FC900356E0F4042C8EE4
:10152800048F05FF123F3F900355E02DFD50010C3D
:101538008C2A8D2B802C900355E0FE900354E0F408
:10154800042E8544F0A4FFAEF0900356E08E048F7D
:1015580005FF123F3F900354E02DFD50010C8C2AEB
:101568008D2BE550C3955F502FE550C395555028F6
:10157800AE22AF23AC2AAD2BEFD39DEE9C4019E5EC
:101588005075F040A4FFAEF090031F12001EE0A8B3
:1015980028B800069529400280037550029000493A
:1015A800E0B40106E550640160028003755002E56D
:0D15B8005065516005C207755900756C0043
:10266F00020FD302112D0212E002132D02140202E7
:02267F0014D86D
:1015C500900050E02402A822B80007D395234002DA
:1015D500C207900025E0B40109900059E0C39403C7
:1015E500400302174B900049E0600302169BE5504B
:1015F500D394014034E55075F040A4FFAEF090035C
:101605001412001EE0A822B8001FD39523401AE546
:101615005075F040A4FFAEF090031F12001EE0A825
:1016250028B80005D39529500280021550E550D3FE
:101635009401402FE55075F040A4FFAEF0900312E1
:1016450012001EE0C39544501AE55075F040A4FF02
:10165500AEF090031E12001EE0A828B80005D39531
:1016650029500280021550E550D394014021E550E0
:10167500D39555401AE55075F040A4FFAEF09003A0
:101685001E12001EE0A828B80005D3952950028037
:10169500021550021740E550D394024034E55075C9
:1016A500F040A4FFAEF090031412001EE0A822B88B
:1016B500001FD39523401AE55075F040A4FFAEF006
:1016C50090031F12001EE0A828B80005D3952950E5
:1016D5000280021550E550D39402402FE55075F075
:1016E50040A4FFAEF090031212001EE0C3954450D3
:1016F5001AE55075F040A4FFAEF090031E12001ECF
:10170500E0A828B80005D39529500280021550E5B8
:1017150050D394024021E550D39555401AE55075B4
:10172500F040A4FFAEF090031E12001EE0A828B8FA
:101735000005D39529500280021550E5506551608A
:1017450005C207755900900060E0D3954450099093
:101755000054E0C395445002C207900059E070035D
:101765000219AEA2A5B34008A2A4B340030219977B
:10177500AE34AF357441D39F749C9E4005783412C6
:10178500003FAE34AF35EFB48806EEB413028003E4
:10179500021974A2A55003021837900059E0B4014C
:1017A5000B90004FE0D3955F4002055F900059E034
:1017B500B40253E55075F040A4FFAEF0900320123B
:1017C500001EE0C39559503E90004FE0D395504020
:1017D50020E550C395555019E55075F040A4FFAE6E
:1017E500F090031412001EE0A822B80006952340CD
:1017F500028002055090004FE0F55FE550655160AD
:1018050005C207755900900059E0B4032590004FB3
:10181500E0D395504007E550C39555400280020539
:101825005090004FE0F55FE55065516005C20775C2
:101835005900A2A45003021974900059E0B4016E36
:10184500900049E07035E550D394014029E5507585
:10185500F040A4FFAEF090031E12001EE0A828B8C9
:10186500000FD39529400A155075590085505F80A2
:101875000385505F8003755F018033E550D3940283
:101885004029E55075F040A4FFAEF090031E12000C
:101895001EE0A828B8000FD39529400A15507559A0
:1018A5000085505F800385505F8003755F0290005F
:1018B50059E0D394015003021968E55075F040A42E
:1018C500FFAEF090032012001EE0C39559400302BD
:1018D5001968900049E07041E550D394014034E522
:1018E5005075F040A4FFAEF090031112001EE0A861
:1018F50022B8001FD39523401AE55075F040A4FF88
:10190500AEF090031E12001EE0A828B80005D3957E
:1019150029500280021550803FE550D3940240348F
:10192500E55075F040A4FFAEF090031112001EE0E3
:10193500A822B8001FD39523401AE55075F040A49E
:10194500FFAEF090031E12001EE0A828B80005D3D4
:101955009529500280021550E55065516005C20772
:10196500755900E555B40704055D8003755D00E50F
:1019750062B4010EAE34AF35EF64407005EE649C81
:101985006002800EA2A54003755701A2A44003750D
:101995005702A2A5B3B35006A2A4B3B34002800672
:1019A500753500753400021A9CA2A5B34008A2A49F
:1019B500B34003021A88AE34AF357441D39F749C8B
:1019C5009E4005783412003FAE34AF35EFB488063B
:1019D500EEB413028003021A88A2A5406F90006836
:1019E500E0605A90004AE0B4010790004AE4F080B4
:1019F5000690004A7401F090004AE07005755F0397
:101A05008003755F0490004AE0B40104D297800218
:101A1500C297E550B4041AE55075F040A4FFAEF046
:101A250090031E12001EE0A828B80005D395295082
:101A3500028008755003C2077559008003755F045D
:101A4500E555B40704055D8003755D00A2A4403328
:101A5500900069E06021900049E0B40107900049D9
:101A6500E4F080069000497401F0900049E0B4016B
:101A750004D2A08002C2A0E555B40704055D800329
:101A8500755D00A2A5B3B35006A2A4B3B34002800E
:101A950006753500753400E5576558600690008277
:101AA500E06003021C24C29C751400751300C2CAB1
:101AB500E557902681F82828738012122D01800D94
:0D1AC500122DDA8008122EB38003122F8C30
:0F268100021ABE021AC0021AC5021ACA021ACFE2
:101AD200900029E090007AF0E565900057F0E56704
:101AE200900062F0E568900063F0E569900074F0A0
:101AF200E56490007CF0E56690007DF0E56390007F
:101B020080F0E562900081F090002AE090013AF0C6
:101B120090002BE090013BF090002CE090013CF013
:101B2200900041E0900090F0900042E0900091F02F
:101B3200900043E0900092F0900044E0900093F017
:101B4200900045E0900094F0900046E0900095F0FF
:101B5200900047E0900096F0900048E0900097F0E7
:101B6200900033E0900099F0900034E090009AF0F9
:101B7200900035E090009BF0900036E090009CF0E1
:101B82007400900082F0745A900125F0744690011E
:101B920026F07420900127F07434900128F07448E4
:101BA200900129F0745090012AF0743290012BF0C8
:101BB200743490012CF0742090012DF07435900152
:101BC2002EF0742D90012FF07453900130F0746F49
:101BD200900131F0746C900132F07420900133F076
:101BE2009003D4E0900414F0743A90074EF074FD20
:101BF20090074FF01200C9900004E4F0A3F09000A7
:101C0200067475F0A37430F09000087475F0A37434
:101C120030F0855758D2CA754B00D29C741B900085
:101C220023F0E555C394065005E550B5510280678F
:101C3200C207E55075F040A4FFAEF09003221200F7
:101C42001EE030E003D38001C39293E55075F0406B
:101C5200A4FFAEF090032312001EE030E003D38015
:101C620001C39294E55075F040A4FFAEF0900324B6
:101C720012001EE030E003D38001C39291855051DF
:101C8200AE28AF297405BE00039F5007E544D394E4
:101C92000550028002D290E555D394055003021DEF
:101CA200A3C207E550D394014073E55075F040A4F8
:101CB200FFAEF090031E12001EE0A828B80007D362
:101CC200952940021550E5506551604EE55075F07A
:101CD20040A4FFAEF090032212001EE030E003D3D6
:101CE2008001C39293E55075F040A4FFAEF09003DB
:101CF2002312001EE030E003D38001C39294E5502A
:101D020075F040A4FFAEF090032412001EE030E014
:101D120003D38001C39291855051021DA3E555B4AE
:101D220006279000ACE030E003D38001C392939089
:101D320000ADE030E003D38001C392949000AEE0A6
:101D420030E003D38001C39291E555B40727900098
:101D5200A5E030E003D38001C392939000A6E03067
:101D6200E003D38001C392949000A7E030E003D354
:101D72008001C39291E555B4082790009EE030E0BF
:101D820003D38001C3929390009FE030E003D3809D
:101D920001C392949000A0E030E003D38001C3928B
:101DA20091900072E06058E54475F00284FF7E0075
:101DB20090014E12001EE0F55BE54675F00A84FFC5
:101DC2007E0090024E12001EE0F55CE55B255CD3BE
:101DD2009464400BE55B255CC39464F55B800375FA
:101DE2005B00E55B75F00284FF7E008F5BEFC394BE
:101DF200335007EF24CDF55B8003755BFF801CE554
:101E02004475F00284FF7E0090014E12001EE075C0
:101E1200F00284FF7E00EF24CDF55BE595C3955B70
:101E22004004C2928002D292A207B34005E555B4A3
:101E320007037570CDE595C395704004C287800293
:101E4200D287E542C394064003022447A2EDB35071
:101E520003022447C2EDE5426003021FA97E017F0F
:101E620000E5BE123F5DE5BD2FFF50010E90000060
:101E7200EEF0A3EFF0900029E0B401177E0F7FFF90
:101E8200900000E0FCA3E0FD120003900000EEF0E1
:101E9200A3EFF0900079E0B4025B900000E0FEA3B3
:101EA200E0FF90000AE0FCA3E0FDEDD39FEC9E4032
:101EB2000F900000E0F8A3E090000AC8F0A3C8F079
:101EC200900000E0FEA3E0FF90000CE0FCA3E0FD28
:101ED200EFD39DEE9C400F900000E0F8A3E090004D
:101EE2000CC8F0A3C8F0900000E0FEA3E0FF740469
:101EF200123F4F8F43900079E07060900000E0FE47
:101F0200A3E0FF90000AE0FCA3E0FDEFD39DEE9C6E
:101F1200400D120003900000EEF0A3EFF080079056
:101F22000000E4F0A3F0900000E0FEA3E0FF7410D4
:101F3200123F5D900026E08E048F05FF123F3F9016
:101F42000000ECF0A3EDF07400D39D74019C4008F6
:101F5200900001E0F54380037543FFE54375F00A05
:101F6200A4FFAEF074198E048F05FF123F3F8D441B
:101F7200ED2531FFAE3050010E7401123F4F8F44F8
:101F8200854431753000EFD394624003754462900A
:101F92000072E064016006900066E06002800575F0
:101FA2004201800375BB17E542B40102800302209F
:101FB200997E017F00E5BE123F5DE5BD2FFF500116
:101FC2000E900000EEF0A3EFF0900072E0B4017EFC
:101FD200E53345326025AC32AD331DBDFF011C8FA8
:101FE200028E038C068D07903A9312002EE493FE24
:101FF200740193FFEFC39AEE9B4002800578321280
:102002003F87AE32AF3374B3BE0025D39F402190D9
:102012000000E0FCA3E0FD0FBF00010E903A931216
:10202200002EE493FE740193FFEDC39FEC9E4002E9
:102032008005783212003FAE32AF33E569123F5D60
:1020420074648E048F05FF123F3F8D4680339000EB
:1020520066E0602D900000E0FEA3E0FFEFD3940065
:10206200EE9408400F900066E0B40104C2098002B9
:10207200D209800D900066E0B40104D2098002C248
:1020820009900072E064026006900066E0600575E7
:10209200BB168003754202E542B4020280030221AC
:1020A200877E017F00E5BE123F5DE5BD2FFF500137
:1020B2000E900000EEF0A3EFF0900072E0B4027E0A
:1020C200E53345326025AC32AD331DBDFF011C8FB7
:1020D200028E038C068D07903BFD12002EE493FEC8
:1020E200740193FFEFC39AEE9B400280057832128F
:1020F2003F87AE32AF3374B3BE0025D39F402190E9
:102102000000E0FCA3E0FD0FBF00010E903BFD12BA
:10211200002EE493FE740193FFEDC39FEC9E4002F8
:102122008005783212003FAE32AF33E569123F5D6F
:1021320074648E048F05FF123F3F8D4680339000FA
:1021420066E0602D900000E0FEA3E0FFEFD3940074
:10215200EE9408400F900066E0B40104C2098002C8
:10216200D209800D900066E0B40104D2098002C257
:1021720009900072E07003754600900066E07002FC
:10218200C20975BB1FE542B403457E017F00E5BE6F
:10219200123F5DE5BD2FFF50010E900000EEF0A34F
:1021A200EFF07409123F5D74E68E048F05FF123F53
:1021B2003F8C408D41E5492DFD50010C74018C0688
:1021C2008D07123F4F8E408F4185414975BB19E5FE
:1021D20042B40402800302232F7E017F00E5BE1277
:1021E2003F5DE5BD2FFF50010E900000EEF0A3EF22
:1021F200F07404123F4F8F4AE563B4010280030278
:1022020022BC756A00756A00E56AD394074003022E
:1022120022A9E56A900041123F75E0D3954A501A0F
:10222200E56A900041123F75E0F404254AFEE56A32
:10223200900037123F75EEF08017E56A9000411268
:102242003F75E0C3954AFEE56A900037123F75EE8E
:10225200F0E56AC394044009900084E0C3956A5093
:102262003BE56A6029E56A900037123F75FEE0FFA0
:10227200EE90003FE0D39F4013E56A900037123F93
:1022820075E090003FF0E56A900040F0800E90000B
:1022920037E090003FF07400900040F0786A7401DB
:1022A20026F6400302220A900040E0F4042408F5D6
:1022B20055E555D394054002C290E563D39401409D
:1022C2002FE54AD3946E4004D20D8002C20D75559B
:1022D20005E563B40205A20DB340028003755507FC
:1022E200E563B40306A20DB3B3400280037555073C
:1022F200E55665556008E55004F551855556E55596
:10230200B40708E5B54480F5B58006E5B5547FF518
:10231200B5E55564066005E555B40808E5B5441011
:10232200F5B58006E5B554EFF5B575BB13E542B4D6
:10233200050280030224437E017F00E5BE123F5D59
:10234200E5BD2FFF50010E900000EEF0A3EFF074F8
:1023520004123F4F8F45E562B4020280030224401B
:10236200756A00756A00E56AD3940340030223F795
:10237200E56A900033123F75E0D39545501AE56A3D
:10238200900033123F75E0F4042545FEE56A9000A3
:102392002D123F75EEF08017E56A900033123F75FB
:1023A200E0C39545FEE56A90002D123F75EEF0E51B
:1023B2006A6029E56A90002D123F75FEE0FFEE90FB
:1023C2000031E0D39F4013E56A90002D123F75E083
:1023D200900031F0E56A900032F0800E90002DE01E
:1023E200900031F07400900032F0786A740126F6A1
:1023F2004003022368900082E07043E5294528608B
:1024020036E557C39403500A900032E004C39403A4
:1024120040028007900032E004F557E557D394025A
:10242200400A900032E004D39402500280079000E8
:1024320032E004F5578007900032E004F55775BB8F
:10244200180542D2ECE55DD3940450030225487589
:10245200CF01C292AE34AF357488D39F74139E40BD
:1024620005A2A5B34014AE34AF357488D39F74135C
:102472009E4005A2A4B340028048783412003FAEC9
:1024820034AF35EFB4883BEEB41337A2A5B350098D
:1024920090004FE0D395505002800405508011A265
:1024A200A5B3500890004FE0655060028002D20749
:1024B200A2A4B35007E550D39401500280041550F2
:1024C200C207A2A5B3B35006A2A4B3B340028006CA
:1024D200753500753400E5506551604EE55075F074
:1024E20040A4FFAEF090032212001EE030E003D3BE
:1024F2008001C39293E55075F040A4FFAEF09003C3
:102502002312001EE030E003D38001C39294E55011
:1025120075F040A4FFAEF090032412001EE030E0FC
:1025220003D38001C39291855051A2074005757073
:10253200CD80037570FFE595C395704004C2878016
:1025420002D287022451AE24AF25EFD39420EE9419
:102552004E5003022643120481C28E758D00758B84
:1025620000754B00D28EC207756F00756E007570D4
:10257200CD755004752300752200755300755900FE
:10258200C296900059E06004D2958002C2959000F4
:102592004AE0B40104D2978002C297900049E0B4A5
:1025A2000104D2A08002C2A0A209B34004D2A28038
:1025B20002C2A290006BE0601812371CA200B34066
:1025C20008E5B54408F5B58006E5B554F7F5B580DC
:1025D20002C20090006EE06018123871A202B3408D
:1025E20008E5B54402F5B58006E5B554FDF5B580BC
:1025F20006E5B554FDF5B590000E74FDF0A374E840
:10260200F0E542B40603754200900025E4F075251A
:1026120000752400758D00758B00754B00900024A9
:10262200E0C394035008900024E004F08006740391
:10263200900024F0900024E0B40306E5B554FEF5C2
:10264200B5AE26AF27EFD39410EE9427401CC2CA32
:1026520075CD0075CC00752700752600D2CA754D60
:0D26620000752900752800755400020CAEAB
:103A230000000100013201640196019602000212B6
:103A330002240200020003000340038003C00400C9
:103A43000440048004C005000600060006000600CA
:103A5300060006000600060000FF01310163019520
:103A630001FF01FF0211022302FF02FF02FF033FD6
:103A7300037F03BF03FF043F047F04BF04FF05FF6D
:103A830006FF06FF06FF06FF06FF06FF06FF06FF0B
:103A93000FAA0FA50F9F0F9A0F940F8D0F870F80FB
:103AA3000F780F710F680F600F570F4E0F450F3BC5
:103AB3000F300F250F1A0F0E0F020EF50EE80EDB57
:103AC3000ECC0EBE0EAE0E9F0E8E0E7D0E6C0E5ADB
:103AD3000E470E340E200E0C0DF70DE20DCB0DB577
:103AE3000D9D0D850D6D0D540D3A0D200D050CE941
:103AF3000CCE0CB10C940C760C580C3A0C1B0BFB33
:103B03000BDB0BBB0B9A0B790B570B350B130AF122
:103B13000ACE0AAB0A870A640A400A1C09F809D4C8
:103B230009B0098C09670943091F08FB08D608B2C5
:103B3300088E086A0846082307FF07DC07B90796BB
:103B430007730751072F070D06EC06CA06AA068955
:103B530006690649062A060A05EC05CD05B0059255
:103B630005750558053C0520050504EA04CF04B591
:103B7300049C04820469045104390422040B03F4F1
:103B830003DE03C803B2039D038903750361034D79
:103B9300033B03280316030402F202E102D102C02D
:103BA30002B002A002910282027302650257024927
:103BB300023C022F02220216020901FD01F201E674
:103BC30001DB01D001C601BB01B101A7019D019435
:103BD300018B018201790170016801600158015074
:103BE3000148014101390132012B0125011E011850
:103BF3000111010B010500FF00FA0FA60FA00F9999
:103C03000F920F8B0F840F7C0F740F6B0F620F5883
:103C13000F4E0F430F380F2C0F1F0F120F050EF708
:103C23000EE80ED80EC80EB70EA50E930E800E6CBE
:103C33000E580E420E2C0E150DFD0DE40DCB0DB1DD
:103C43000D950D790D5D0D3F0D200D010CE10CC09F
:103C53000C9E0C7C0C590C350C100BEA0BC40B9E00
:103C63000B760B4F0B260AFD0AD40AAA0A800A55C3
:103C73000A2A09FF09D409A8097C0950092508F96A
:103C830008CD08A10875084A081E07F307C8079D51
:103C930007730749072006F706CE06A6067E0657D2
:103CA3000630060A05E405BF059B05770554053272
:103CB300051004EF04CE04AE048F047104530435DD
:103CC300041903FD03E203C703AD0394037B0363FA
:103CD300034B0334031E030802F302DE02CA02B6D7
:103CE30002A30291027F026D025C024C023C022C91
:103CF300021D020E020001F201E401D701CA01BE56
:103D030001B101A6019A018F0185017A0170016653
:103D1300015D0153014A01410139013101290121A9
:103D230001190112010B010400FD00F700F000EA84
:103D330000E400DE00D900D300CE00C900C400BFF8
:103D430000BA00B500B100AD00A800A400A0009C1B
:103D5300009900950091008E008A008700840081FD
:043D6300007E007B63
:10269000751A00751900AE19AF1AAC17AD18EDC355
:1026A0009FEC9E401674FF123F2F75CF01781A746D
:1026B0000126F6500418E436F650DB22900786E433
:1026C000F0A3F0751000750F00751300751400C2AB
:1026D0000ED20F22C2AF75D900758F0375B7A575DD
:1026E000B7F190F800E4F0758F0175B7A575B7F1F3
:1026F000E50890F800F075B7A575B7F190F801E41A
:10270000F075B7A575B7F190079DE090F802F075E8
:10271000B7A575B7F19007A1E090F803F075B7A5DC
:1027200075B7F190079EE090F804F075B7A575B7FE
:10273000F190079FE090F805F075B7A575B7F19097
:1027400007A0E090F806F075B7A575B7F19007A25D
:10275000E090F807F0758F0075D940D2AF2290074E
:1027600088E0B4AB61C2AF75D90075B62275F522A9
:10277000758F0375B7A575B7F1740090F600F07505
:102780008F01750A00750900AE09AF0A7413BE0007
:10279000279F402475B7A575B7F190078912001ED1
:1027A000E0FC90F60012001EECF0780A740126F6A8
:1027B000500418E436F650D0758F0075F51175B6D3
:1027C0002075D940D2AF22C2AF75D90075F52275F8
:1027D0000A00750900AE09AF0A7413BE00229F40BB
:1027E0001F90F60012001EE493FC90078912001E51
:1027F000ECF0780A740126F6500418E436F650D549
:1028000075F51175D940D2AF22900788E0B4AA02BD
:102810008003022946C2AF75D90075B62275F5222C
:10282000758F0375B7A575B7F1740090EE00F0755C
:10283000B7A575B7F1740090F000F075B7A575B73E
:10284000F1740090F200F075B7A575B7F1740090BF
:10285000F400F0758F01750A00750900AE09AF0A22
:1028600074FFC39F74019E402475B7A575B7F1909E
:10287000004E12001EE0FC90EE0012001EECF078FC
:102880000A740126F6500418E436F650CF750A0093
:10289000750900AE09AF0A74FFC39F74019E4024FE
:1028A00075B7A575B7F190024E12001EE0FC90F0CE
:1028B0000012001EECF0780A740126F6500418E4A9
:1028C00036F650CF750A00750900AE09AF0A74FFDD
:1028D000C39F74019E402475B7A575B7F190044E4F
:1028E00012001EE0FC90F20012001EECF0780A7458
:1028F0000126F6500418E436F650CF750A00750923
:1029000000AE09AF0A74FFC39F74019E402475B7DF
:10291000A575B7F190064E12001EE0FC90F400126F
:10292000001EECF0780A740126F6500418E436F61E
:1029300050CF758F0075F51175B62075D940D2AF9F
:10294000743A90074EF022900788E0B4AA02800300
:10295000022A84C2AF75D90075B62275F522758F2B
:102960000375B7A575B7F1740090E600F075B7A5CB
:1029700075B7F1740090E800F075B7A575B7F174FC
:102980000090EA00F075B7A575B7F1740090EC00FF
:10299000F0758F01750A00750900AE09AF0A74FF62
:1029A000C39F74019E402475B7A575B7F190004E82
:1029B00012001EE0FC90E60012001EECF0780A7493
:1029C0000126F6500418E436F650CF750A00750952
:1029D00000AE09AF0A74FFC39F74019E402475B70F
:1029E000A575B7F190024E12001EE0FC90E80012AF
:1029F000001EECF0780A740126F6500418E436F64E
:102A000050CF750A00750900AE09AF0A74FFC39F65
:102A100074019E402475B7A575B7F190044E12005D
:102A20001EE0FC90EA0012001EECF0780A74012609
:102A3000F6500418E436F650CF750A00750900AE5A
:102A400009AF0A74FFC39F74019E402475B7A57532
:102A5000B7F190064E12001EE0FC90EC0012001E32
:102A6000ECF0780A740126F6500418E436F650CFDC
:102A7000758F0075F51175B62075D940D2AF743ACF
:102A800090074EF022900788E0B4AA028003022B40
:102A9000C2C2AF75D90075B62275F522758F037560
:102AA000B7A575B7F1740090DE00F075B7A575B7DE
:102AB000F1740090E000F075B7A575B7F17400905F
:102AC000E200F075B7A575B7F1740090E400F075F9
:102AD0008F01750A00750900AE09AF0A74FFC39F24
:102AE00074019E402475B7A575B7F190004E120091
:102AF0001EE0FC90DE0012001EECF0780A74012645
:102B0000F6500418E436F650CF750A00750900AE89
:102B100009AF0A74FFC39F74019E402475B7A57561
:102B2000B7F190024E12001EE0FC90E00012001E71
:102B3000ECF0780A740126F6500418E436F650CF0B
:102B4000750A00750900AE09AF0A74FFC39F7401CE
:102B50009E402475B7A575B7F190044E12001EE093
:102B6000FC90E20012001EECF0780A740126F65088
:102B70000418E436F650CF750A00750900AE09AFA7
:102B80000A74FFC39F74019E402475B7A575B7F101
:102B900090064E12001EE0FC90E40012001EECF0C5
:102BA000780A740126F6500418E436F650CF758F73
:102BB0000075F51175B62075D940D2AF743A9007FB
:102BC0004EF022900788E0B4AA028003022D00C2D2
:102BD000AF75D90075B62275F522758F0375B7A547
:102BE00075B7F1740090D600F075B7A575B7F1749C
:102BF0000090D800F075B7A575B7F1740090DA00B1
:102C0000F075B7A575B7F1740090DC00F0758F0111
:102C1000750A00750900AE09AF0A74FFC39F7401FD
:102C20009E402475B7A575B7F190004E12001EE0C6
:102C3000FC90D60012001EECF0780A740126F650C3
:102C40000418E436F650CF750A00750900AE09AFD6
:102C50000A74FFC39F74019E402475B7A575B7F130
:102C600090024E12001EE0FC90D80012001EECF004
:102C7000780A740126F6500418E436F650CF750A27
:102C800000750900AE09AF0A74FFC39F74019E402E
:102C90002475B7A575B7F190044E12001EE0FC90A4
:102CA000DA0012001EECF0780A740126F6500418BF
:102CB000E436F650CF750A00750900AE09AF0A7404
:102CC000FFC39F74019E402475B7A575B7F19006A8
:102CD0004E12001EE0FC90DC0012001EECF0780AA0
:102CE000740126F6500418E436F650CF758F00753F
:102CF000F51175B62075D940D2AF743A90074EF0F1
:102D000022C2AF75D90075F522750A00750900AEAB
:102D100009AF0A74FFC39F74019E401F90EE00121A
:102D2000001EE493FC90004E12001EECF0780A7432
:102D30000126F6500418E436F650D4750A007509D9
:102D400000AE09AF0A74FFC39F74019E401F90F04C
:102D50000012001EE493FC90024E12001EECF0786C
:102D60000A740126F6500418E436F650D4750A00A9
:102D7000750900AE09AF0A74FFC39F74019E401F1E
:102D800090F20012001EE493FC90044E12001EEC20
:102D9000F0780A740126F6500418E436F650D4751B
:102DA0000A00750900AE09AF0A74FFC39F74019E43
:102DB000401F90F40012001EE493FC90064E120097
:102DC0001EECF0780A740126F6500418E436F6502A
:102DD000D475F51175D940D2AF22C2AF75D900753F
:102DE000F522750A00750900AE09AF0A74FFC39F8A
:102DF00074019E401F90E60012001EE493FC9000B8
:102E00004E12001EECF0780A740126F6500418E405
:102E100036F650D4750A00750900AE09AF0A74FF82
:102E2000C39F74019E401F90E80012001EE493FCB3
:102E300090024E12001EECF0780A740126F650043F
:102E400018E436F650D4750A00750900AE09AF0AC9
:102E500074FFC39F74019E401F90EA0012001EE49D
:102E600093FC90044E12001EECF0780A740126F6D2
:102E7000500418E436F650D4750A00750900AE09FE
:102E8000AF0A74FFC39F74019E401F90EC001200B4
:102E90001EE493FC90064E12001EECF0780A7401BA
:102EA00026F6500418E436F650D475F51175D9405D
:102EB000D2AF22C2AF75D90075F522750A00750927
:102EC00000AE09AF0A74FFC39F74019E401F90DEDD
:102ED0000012001EE493FC90004E12001EECF078ED
:102EE0000A740126F6500418E436F650D4750A0028
:102EF000750900AE09AF0A74FFC39F74019E401F9D
:102F000090E00012001EE493FC90024E12001EECB2
:102F1000F0780A740126F6500418E436F650D47599
:102F20000A00750900AE09AF0A74FFC39F74019EC1
:102F3000401F90E20012001EE493FC90044E120029
:102F40001EECF0780A740126F6500418E436F650A8
:102F5000D4750A00750900AE09AF0A74FFC39F74E7
:102F6000019E401F90E40012001EE493FC90064E68
:102F700012001EECF0780A740126F6500418E436AC
:102F8000F650D475F51175D940D2AF22C2AF75D9BC
:102F90000075F522750A00750900AE09AF0A74FFC5
:102FA000C39F74019E401F90D60012001EE493FC44
:102FB00090004E12001EECF0780A740126F65004C0
:102FC00018E436F650D4750A00750900AE09AF0A48
:102FD00074FFC39F74019E401F90D80012001EE42E
:102FE00093FC90024E12001EECF0780A740126F653
:102FF000500418E436F650D4750A00750900AE097D
:10300000AF0A74FFC39F74019E401F90DA00120044
:103010001EE493FC90044E12001EECF0780A74013A
:1030200026F6500418E436F650D4750A00750900E7
:10303000AE09AF0A74FFC39F74019E401F90DC006D
:1030400012001EE493FC90064E12001EECF0780A6B
:10305000740126F6500418E436F650D475F511754F
:10306000D940D2AF22E51464046006E59964FF609C
:10307000028031A20E4004D20E8027E5146008744D
:10308000E62514900023F0E513600874F0251390F2
:103090000023F0E514B4010280FE751400751300DE
:1030A000C20E8002C20EE5149039C6F82828737546
:1030B0001400E599B4FF03751301E599B4FE037597
:1030C0001302E599B4FD03751303E599B4FC037588
:1030D0001304E599B4FA03751305E599B4FB067575
:1030E0001401120481E599B4F906751404120481DF
:1030F000E599D394E54007E599C394F04002801622
:103100008599157514027E017F00E515C394E612BA
:103110003F5D8E0D8F0E900786E4F0A3F0E599D306
:1031200094C44007E599C394E64002802885991528
:1031300075140374E5C39515F50E750D00AE0DAF4E
:103140000E903A2312002EE493F8740193900786B0
:10315000C8F0A3C8F0D2990235DA900786E0FEA342
:10316000E0FFEFC39400EE94054009EFD394FFEE27
:1031700094064013900786E0FEA3E0FF90004E12F5
:10318000001EE599F0800385996B90078612000E6A
:10319000900786E0FEA3E0FFEFB40106EEB407025D
:1031A00080030233E790074EE0B43C028003023311
:1031B000E775FFA0A20AB35005A20BB34003023289
:1031C000DAC29C90007AE090078CF0900057E09073
:1031D000078DF0900062E090078EF0900063E09021
:1031E000078FF0900074E0900790F090007CE090E2
:1031F0000791F090007DE0900792F0900080E090C1
:103200000793F0900081E0900794F090013AE090ED
:103210000795F090013BE0900796F090013CE0901C
:103220000797F0900090E0900798F0900091E09060
:103230000799F0900092E090079AF0900093E09048
:10324000079BF0900094E090079CF0900095E09030
:10325000079DF0900096E090079EF0900097E09018
:10326000079FF0900099E09007A0F090009AE090FE
:1032700007A1F090009BE09007A2F090009CE090E6
:1032800007A3F07400900082F01200C974AB90079D
:0D32900088F012275E74AA900788F0E557B9
:0639C6000230AF02315A8D
:10329D009039E7F82828738012122809800D122919
:0B32AD00478008122A858003122BC303
:0F39E7000232A40232A60232AB0232B00232B573
:1032B800900788E4F090013AE0700C90013BE070D0
:1032C8000690013CE060028004C20A8002D20A0231
:1032D80033DCC29C900078E0900789F090005EE0B3
:1032E80090078AF090005FE090078BF090007AE0FA
:1032F80090078CF0900057E090078DF0900062E006
:1033080090078EF0900063E090078FF0900074E0D3
:10331800900790F090007CE0900791F090007DE09D
:10332800900792F0900080E0900793F0900081E081
:10333800900794F090013AE0900795F090013BE0F7
:10334800900796F090013CE0900797F0900090E08D
:10335800900798F0900091E0900799F0900092E023
:1033680090079AF0900093E090079BF0900094E00B
:1033780090079CF0900095E090079DF0900096E0F3
:1033880090079EF0900097E090079FF0900099E0DA
:103398009007A0F090009AE09007A1F090009BE0C1
:1033A8009007A2F090009CE09007A3F074009000B2
:1033B80082F074AB900788F012275E74AA90078891
:1033C800F0122809122947122A85122BC3D29C759C
:1033D80099FB80FED29C7514007513007599FB0249
:1033E80035DA900786E0FEA3E0FFEF4E7006859978
:1033F80010750F00900786E0FEA3E0FF74016F4E82
:10340800701BAC0FAD10AA0DAB0EED2BFBEC3AFA0E
:103418008A068B0790004E12001EE599F0900786E9
:1034280012000E900786E0FEA3E0FF74026F4E7054
:103438000C1200C98515997514007513000235DA48
:10344800900786E0FEA3E0FF90004E12001EE5996B
:10345800F090078612000E900786E0FEA3E0FFAC0E
:103468000DAD0E8F028E038C068D07903A5B12000D
:103478002EE493F9740193FEEAD39EEB99400985F3
:1034880015997514007513000235DA900786E0FE69
:10349800A3E0FF90004E12001EE599F090078612F7
:1034A800000E900786E0FEA3E0FFEFB40006EEB43E
:1034B800010280030235DA75FFA090001CE0D39466
:1034C800C7400B90001CE0C394C8F516801A900002
:1034D8001CE0D39463400B90001CE0C39464F51681
:1034E800800690001CE0F516E51675F002A4FFAE04
:1034F800F08F6AEF90004E123F75EFFCE0FDEC9004
:103508000051123F75EDFCE0FDEC2DB5160280036D
:103518000235CC0FEF90004E123F75E56AFFE0FCD4
:10352800EF900052123F75ECFFE0FCEFC39CB5161C
:103538000280030235CCE56A900050123F75E56AB7
:10354800FFE0FCEF900053123F75ECFFE0FCEF2C1E
:10355800B51671E56A900054123F75E0C395169050
:10356800079DF0E56A900055123F75E0C3951690E7
:10357800079EF0E56A900058123F75E0C3951690D3
:10358800079FF0E56A900059123F75E0C3951690C1
:1035980007A0F0E56A90005A123F75E0C3951690AF
:1035A80007A1F0E56A90005B123F75E0C39516909D
:1035B80007A2F01226D47599F975186475170012C8
:1035C800269080FE7599FF7518647517001226906D
:0235D80080FE73
:0939CC000233EA0234480234938C
:1035DA0022E5139039D5F828287302371B900786FD
:1035EA00E0FEA3E0FF90001212001EE0F59990079A
:1035FA008612000E900786E0FEA3E0FF74116F4E5C
:10360A00700375130002371B85619902371B9007F7
:10361A0086E0FEA3E0FF90004E12001EE0F599EF4F
:10362A00B40107EEB4070375130090078612000E63
:07363A0002371B900787E037
:0F39D5000235E40235E702361202361802363D9B
:103641009039F6F82828738523990237108529992E
:103651000237108543990237108546990237108544
:103661005099023710855F990237108555990237B5
:1036710010855799023710756D00900069E070064A
:10368100900068E060028016A2A44006E56D440443
:10369100F56DA2A54006E56D4402F56D801A900016
:1036A1004AE0B40106E56D4410F56D900049E0B4BF
:1036B1000106E56D4420F56DA207B34006E56D44B2
:1036C10001F56DA209B34006E56D4408F56D856D00
:1036D10099803CA20FB340077599FAC20F8017A2D7
:1036E1000CB3400575990F800B900023E0F599907C
:1036F1000023E4F0C20C80178541998012854A9914
:0F370100800D85459980087599FC80037513002C
:1039F60002364802364E02365402365A0236600203
:103A0600366602366C0236720236780236D40236D2
:0D3A1600F90236FE02370302370802370DB1
:0B37100090078612000E800312004894
:0339E4000237188F
:10371B002290006BE0B4010385231190006BE0B4A1
:10372B00020385291190006BE0B4030385431190CC
:10373B00006BE0B4040385461190006BE0B4050305
:10374B0085501190006BE0B4060385551190006B0A
:10375B00E0B4070385571190006CE0FE90006DE01C
:10376B00C39E50030237F290006BE0D39404402CBD
:10377B0090006CE0D39511500990006DE0C395114A
:10378B0050028002D20090006CE0D395115009904A
:10379B00006DE0C395115002C200804990006BE0B0
:1037AB00B4041890006DE0C395115002D200900044
:1037BB006CE0D395114002C200802A90006CE0C3EC
:1037CB009511500990006DE0D3951150028002D2F3
:1037DB000090006CE0D39511500990006DE0C395FB
:1037EB00115002C200807E90006BE0D39404402CF9
:1037FB0090006CE0C39511400990006DE0D39511DA
:10380B0040028002C20090006CE0C3951140099009
:10381B00006DE0D395114002D200804990006BE01F
:10382B00B4041890006CE0C395115002C2009000D4
:10383B006DE0D395114002D200802A90006CE0C35A
:10384B009511400990006DE0D395114002D2009084
:10385B00006CE0D39511400990006DE0C3951140C9
:10386B00028002C2002290006EE0B4010385231196
:10387B0090006EE0B4020385291190006EE0B40352
:10388B000385431190006EE0B4040385461190004C
:10389B006EE0B4050385501190006EE0B40603850D
:1038AB00551190006EE0B4070385571190006FE03F
:1038BB00FE900070E0C39E500302394790006EE00B
:1038CB00D39404402C90006FE0D3951150099000D5
:1038DB0070E0C3951150028002D20290006FE0D3CA
:1038EB0095115009900070E0C395115002C20280EF
:1038FB004990006EE0B40418900070E0C39511502D
:10390B0002D20290006FE0D395114002C202802ACE
:10391B0090006FE0C395115009900070E0D39511A2
:10392B0050028002D20290006FE0D39511500990A3
:10393B000070E0C395115002C202807E90006EE0D1
:10394B00D39404402C90006FE0C395114009900074
:10395B0070E0D3951140028002C20290006FE0C369
:10396B0095114009900070E0D395114002D202806E
:10397B004990006EE0B4041890006FE0C3951150AD
:10398B0002C202900070E0D395114002D202802A4D
:10399B0090006FE0C395114009900070E0D3951132
:1039AB004002D20290006FE0D39511400990007055
:0B39BB00E0C3951140028002C202220E
:093F75002582F582500205832229
:10002E00EF2F500205832582F582E5833E2EF58360
:01003E00229F
:08000300C3EF9DFFEE9CFE22FD
:08003F000806B60002180622B3
:0D000E00A3E004F07006123F6BE004F02246
:083F87000816B6FF021816220D
:0E3F4F00048007C3CE13CECF13CFD5E0F622E9
:103D6700BC000FBE0008ED8FF084FFADF022E4FE2B
:103D7700FF22BE000DEF60FE54F0606F20E70302E4
:103D87003E1DEAC0E0EBC0E078017A0075F001EE75
:103D970020E710EF25E0FFEE33FE0AC5F023C5F05C
:103DA70030E7F0EA5407F9096A7A007B00600108F6
:103DB700C3EC9E40167004ED9F4010ED9FFDEC9EF6
:103DC700FCE5F0CA4ACA03F5F08005E5F003F5F013
:103DD700C3EE13FEEF13FFD9D77908CACBCAD8D0E1
:103DE700EAFEEBFFD0E0FBD0E0FA22EC8FF084FC98
:103DF700ED54F045F0C48FF084FEEDC454F045F067
:103E0700C48FF084FDEEC4FE54F02DFFEE540F3C3A
:103E1700FEADF07C0022790078008FF0EC7E082060
:103E2700E70DC3CD33CD33C933C9C833C8DEF084FA
:103E370049F9E5F08FF0BE00E6FD7C00E9FFE8FEFA
:013E47002258
:0E3F5D00F88FF0A4FFE5F0CE88F0A42EFE222F
:103F2F00600D782B023F39007830D8FED5E0F822AB
:103F3F00EEC0E07E00123D67EFFDEEFCD0E0FE220A
:03000B00023EDED4
:03001B00023EF9A9
:03002B00023F147D
:03000000023F7E3E
:093F7E0075817175D0000207EA9B
:0B001E00E5822FF582E5833EF583228A
:0A3F6B000582D5820215831582221B
:103EDE00C0E0C0F0C083C082C0D075D0001207DF32
:103EEE00D0D0D082D083D0F0D0E032C0E0C0F0C0CD
:103EFE0083C082C0D075D0001207E2D0D0D082D05D
:103F0E0083D0F0D0E032C0E0C0F0C083C082C0D019
:103F1E0075D0001207E5D0D0D082D083D0F0D0E09B
:013F2E003260
:00000001FF
